:100000000C94B9010C94F1010C94F1010C94F101E0
:100010000C94F1010C94F1010C94F1010C94F10198
:100020000C94F1010C94F1010C94E1190C94B31AA5
:100030000C94F3140C94F1010C94F1010C94F10163
:100040000C94F1010C94F1010C94F1010C94F10168
:100050000C94F1010C947B150C94F1010C94F101BA
:100060000C94F1010C94F1010C94F1010C94F10148
:100070000C94F1010C94F1010C94F1010C94F10138
:100080000C94F1010C94F1010C94F1010C94F10128
:100090000C94F1010C94F1010C94F1010C94F10118
:1000A0000C94F1010C94F1010C94F1010904090480
:1000B000350435049D04C805C805C805BB045405AE
:1000C00065056505201B471B3F1C471B3F1C931BF9
:1000D000B61B3F1C0D1C1C1C29003B003D003F00B3
:1000E0004100430045004A004E003A003C003E00FB
:1000F00040004200440068004B004D0035001F00E6
:1001000021002300250027002E00530055001E006B
:1001100020002200240026002D002A005400560052
:100120002B001A0015001C000C00130030005F00AB
:100130006100140008001700180012002F003100A1
:10014000600057003900160009000B000E00330054
:1001500000005C005E00040007000A000D000F00B4
:10016000340028005D000000E1001B0019001100B0
:1001700036003800E50059005B001D000600050050
:1001800010003700000052005A005800E000E20062
:100190002C000000E700E40050004F006300E30083
:1001A000000000000000000000005100620000009C
:1001B0000100010001000100010001000100010037
:1001C0000100010001000100010001000100010027
:1001D0000100010001000100010001000100010017
:1001E0000100010001000100010001000100010007
:1001F00001000100010001000100010001000100F7
:1002000001000100010001000100010001000100E6
:1002100001000100010001000100010001000100D6
:1002200001000100010001000000010001000100C7
:1002300001000100010001000100010001000000B7
:1002400001000100010001000100010001000100A6
:100250000100010001000100010001000000010097
:100260000100010001000100010000000100010087
:10027000010001000100010000000000000000007A
:10028000000001000100000010034200650065004D
:10029000670062006F0079000000120353007700CE
:1002A00069006600740072006100780000000403B9
:1002B000090409023B00020100A0FA090400000140
:1002C00003010100092111010001224000070581FD
:1002D00003080001090401000103000000092111C5
:1002E00001000122320007058203200001120100F3
:1002F0000200000008D804C5EA010001020001055F
:10030000010980A101850319012AB700150126B74B
:1003100000950175108100C0050C0901A10185043B
:1003200019012AA002150126A0029501751081006D
:10033000C005010906A101050719E029E7150025F7
:10034000019508750181029501750881010507195C
:100350000029FF150026FF00950675088100050895
:100360001901290595057501910295017503910102
:10037000C00011241FBECFEFDAE0DEBFCDBF04B650
:1003800003FE18C08091A6029091A702A091A80236
:10039000B091A9028730904BA740B04B59F410920E
:1003A000A6021092A7021092A8021092A902E0E001
:1003B000F8E3099511E0A0E0B1E0E4E9F9E302C057
:1003C00005900D92A838B107D9F722E0A8E8B1E06E
:1003D00001C01D92A63AB207E1F70E94D3110C9416
:1003E000C81C0C94000081E0089581E008950C94ED
:1003F000F50108950C94F9011F93CF93DF9300D07A
:1004000000D01F92CDB7DEB749835A836B833091FA
:100410008B0189819A81311114C0662359F02223FE
:1004200049F00E940108182F682F89819A810E9443
:10043000AA0703C00E94D507182F69817A81812FEE
:1004400004C00E94010869817A810F900F900F907B
:100450000F900F90DF91CF911F910C94250FFC010D
:10046000262F408151816281738184810C94FC012B
:1004700081E00895CF93DF93EC0160E00E942F02AA
:10048000BE01DF91CF910C94FA010C946B100C9487
:10049000671008950E9454060E9449022FEF84E3DA
:1004A0009CE0215080409040E1F700C000000C9497
:1004B000A1150F931F93CF93DF938C0161E00E94EE
:1004C0002F02EC01B8010E94F7018823F1F1B80175
:1004D000CE010E94CC138823C1F1B801CE010E9445
:1004E000E011882391F1B801CE010E9428138823DE
:1004F00061F1F8018281882309F1CB358DE5D807B8
:10050000C1F050F4C115FCE5DF0781F0CF3DDC45BB
:10051000A9F40E94380D19C0CC35EDE5DE0761F075
:10052000CD35DD4559F40E947B0C08C00E944A027B
:100530000CC00E94840C02C00E94870CC801DF918D
:10054000CF911F910F910C94F30180E0DF91CF9137
:100550001F910F9108950E94D5140C94C4020E941B
:10056000C7020C94DB1408950C94B30281E0089543
:100570000C94B6020895CF93C82F0E94B4028C2F1A
:100580000E94B802CF91089580E00C94BB020E94B3
:1005900028140C94BB020E94281490918A01891798
:1005A00021F080938A010C94BB020895CF93DF93CE
:1005B000CDB7DEB72B970FB6F894DEBF0FBECDBF19
:1005C0004F83588769877A878B8761110E94C70B91
:1005D0009E012F5F3F4F86E0F90111928A95E9F75E
:1005E00085E0FE013796D90101900D928A95E1F7D9
:1005F00089819A814C815D81452B31F09F3F31F497
:1006000091E08F3F19F403C091E001C090E090FFAA
:1006100009C049815A816B817C818D819E810E94B4
:10062000E80A05C0C9010E9438028111F2CF2B9659
:100630000FB6F894DEBF0FBECDBFDF91CF91089506
:10064000FC01808191810E9443080895CF93882303
:1006500009F448C0C82F8CEF8C0F813AD0F46C2F6E
:1006600080910201909103010E947714882349F040
:100670006C2F80910201909103010E94AF140E949F
:10068000E90B6C2F80910201909103010E94AD143F
:100690000CC080E28C0F883058F4C77081E001C034
:1006A000880FCA95EAF70E94AA0BCF910C94E90B28
:1006B000EBE5EC0FE33040F4F0E0E15CFE4F8081CD
:1006C00090E0CF910C943F14C85AC73158F4EC2FE6
:1006D000F0E0EE0FFF1FEF5EFE4F80819181CF9122
:1006E0000C945514CF910895882349F1682F8CEF0D
:1006F000860F813A38F480910201909103010E94A3
:10070000AF140CC080E2860F883050F4677081E02F
:1007100001C0880F6A95EAF70E94B00B0C94E90BB0
:100720008BE5860F833020F480E090E00C943F143A
:10073000685A673120F480E090E00C9455140895D5
:100740001F93CF93DF93182FEB010E94260320976E
:1007500041F08FE99FE00197F1F700C00000219779
:10076000F6CF812FDF91CF911F910C9474038933C1
:1007700019F060E070E002C060E570E00C94A00346
:10078000882321F00E94AA0B0C94E90B089588237A
:1007900021F00E94B00B0C94E90B0895CF92DF92E8
:1007A000EF92FF920F931F93CF93DF937C01D62F8D
:1007B000C72FFC011281058102950F700E94A00BCA
:1007C0008823B9F01123A9F08C2F807F803421F089
:1007D00080E28D0F883068F08091640282FD09C04C
:1007E00082E00E94490C0E94A00B91E0D82ED926ED
:1007F00001C0D12CCC2EC2948FE0C8228C2D90E069
:100800008C30910508F0C4C1FC01EA5AFF4F0C94EA
:10081000731C8C2F807FCF70882311F0C295C07F0E
:10082000112399F0CC2309F49FC180E28D0F883009
:1008300010F0D11104C08C2F0E94AA0B03C08C2F82
:100840000E94BA0B0E94E90B8FC18D2F0E94740386
:10085000CC2309F49DC180E28D0F883038F1DD236F
:1008600029F18C2F0E94C00B24C08C2F807FCF7069
:10087000803211F0C295C07FDD2319F0D130A1F193
:100880003DC08091640282FF17C0112349F0CC2340
:1008900029F08C2F0E94AA0B0E94E90B80E065C111
:1008A00080E00E947403CC2309F472C18C2F0E9453
:1008B000B00B0E94E90B6CC1112371F0002341F0D1
:1008C000013031F40E94CA0B8C2B0E94D20B60C104
:1008D0000E94CA0B8C2B1DC0002319F0013009F4B3
:1008E00057C10E94DF0B25C0112321F0063008F00C
:1008F0004FC10EC0053008F04BC11BC0112361F081
:10090000002331F0F701858180FF2EC18F70858330
:100910008C2F0E94C0033CC1002359F0D93309F049
:1009200034C1FFEF07EE13E0F15000401040E1F753
:100930002AC18C2F0E94C7032BC18C2F86958695C8
:10094000837019F0813061F023C1112321F08D2FC4
:100950009C2F937002C080E090E00E943F1420C161
:10096000112321F08D2F9C2F937002C080E090E026
:100970000E94551415C18C2F837009F047C01111C6
:100980000BC12D2F229526952770220F220F6D2F38
:100990006F70862F90E0A0E0B0E0022E04C0880FB8
:1009A000991FAA1FBB1F0A94D2F7D4FF10C04FE0B3
:1009B00050E060E070E004C0440F551F661F771FD1
:1009C0002A95D2F7409550956095709503C040E008
:1009D00050E0BA01C695C695C3708A019B01082BE9
:1009E000192B2A2B3B2BC901B801C23049F058F40E
:1009F000C13019F00E94C006CFC00E94AE06CCC024
:100A00000E94D206C9C00E94AC06C6C0112319F0CC
:100A10008C2F817001C08695882309F4BDC02D2FCD
:100A2000229526952770220F220F6D2F6F70862F2B
:100A300090E0A0E0B0E0022E04C0880F991FAA1F2A
:100A4000BB1F0A94D2F7D4FF10C04FE050E060E023
:100A500070E004C0440F551F661F771F2A95D2F718
:100A6000409550956095709503C040E050E0BA0104
:100A7000C695C695C3708A019B01082B192B2A2B9A
:100A80003B2BC901B801C23049F058F4C13019F00C
:100A90000E94850781C00E9473077EC00E9497074D
:100AA0007BC00E94E60678C0CF70112339F08C2FEE
:100AB0000E940C078D2F0E94C0036EC08D2F0E94D4
:100AC000C7038C2F0E942D0767C0D23F21F128F465
:100AD000D03F41F0D13FC1F043C0D33F19F1D43FE3
:100AE00079F03EC0112341F0053008F051C08C2F41
:100AF0008F710E9452074CC0063008F049C0F7CFF2
:100B00008091640282FF18C0112339F08C2F8F71FD
:100B10000E940C073DC01123C9F38C2F8F710E94D6
:100B20002D0736C0112329F08C2F8F710E94F706F4
:100B30002FC00E94F2062CC0112349F0CF718C2FD8
:100B40000E940C0763E08C2F0E942E0C21C081E0D4
:100B50000E94490C0230E0F082E00E94490C18C06B
:100B6000112331F0002391F28D2F0E94260310C033
:100B7000002399F2D93349F41FEF27EE33E01150E7
:100B800020403040E1F700C000008D2F0E94740328
:100B900088EF8C0D843020F40E9428140E94BB0240
:100BA000DD20C9F00E949C0B80FD15C0F701128268
:100BB0000E94960B0E940C07C7010E940C060E941F
:100BC000960BDF91CF911F910F91FF90EF90DF90E7
:100BD000CF900C942D07DF91CF911F910F91FF9033
:100BE000EF90DF90CF9008950F931F93CF93DF93F3
:100BF000EC01688179818A810E944E088C010E94F3
:100C0000A9070E949A06B801CE010E94CE03DF9187
:100C1000CF911F910F910895CF93DF93EC019881AD
:100C200089812B813C81232B31F08F3F31F481E08E
:100C30009F3F19F403C081E001C080E080FD1DC02A
:100C4000CE010E945902811110C00E94A00B88237E
:100C5000A1F08A81882389F08091640282FD0DC011
:100C600082E0DF91CF910C94490CCE010E94F405F3
:100C7000CE01DF91CF910C943A02DF91CF9108958C
:100C800080E090E00E943F1480E090E00E945514C4
:100C90000E94C70B0C94E90B809102019091030113
:100CA0000E94B1140C9440060E94B70B0C944C06A1
:100CB00092959F70963079F010F4925001C09A503E
:100CC000923068F4803F69F018F4883E40F409C01F
:100CD000843F29F406C0883E20F0813F11F080E077
:100CE000089581E00895FC01808191810E9443086C
:100CF0000E9458060895CF93DF9300D000D01F9232
:100D0000CDB7DEB70F900F900F900F900F90DF913F
:100D1000CF910895CF93DF9300D000D000D0CDB70E
:100D2000DEB726960FB6F894DEBF0FBECDBFDF91BB
:100D3000CF910895089508950C949B060C949C06F9
:100D40000E949E066093D6017093D7018093D801CC
:100D50009093D9010C9440060C94A0060F931F9316
:100D60000091D6011091D7012091D8013091D9017D
:100D7000602B712B822B932B1F910F910C94A0064B
:100D80000F931F930091D6011091D7012091D801A4
:100D90003091D90160237123822393231F910F91F6
:100DA0000C94A0060F931F930091D6011091D701C8
:100DB0002091D8013091D90160277127822793278C
:100DC0001F910F910C94A0060C949B060E94E406C0
:100DD0006093D2017093D3018093D4019093D50195
:100DE0000C94400660E070E0CB010C94E6060F9393
:100DF0001F9341E050E060E070E08A019B0104C075
:100E0000000F111F221F331F8A95D2F7C901B801A5
:100E10001F910F910C94E6060F931F9341E050E051
:100E200060E070E004C0440F551F661F771F8A956D
:100E3000D2F78091D2019091D301A091D401B091C9
:100E4000D5018A019B01082B192B2A2B3B2BC901A9
:100E5000B8011F910F910C94E6060F931F9341E088
:100E600050E060E070E004C0440F551F661F771F1C
:100E70008A95D2F740955095609570958091D201F2
:100E80009091D301A091D401B091D5018A019B0129
:100E9000082319232A233B23C901B8011F910F916D
:100EA0000C94E6060F931F9341E050E060E070E081
:100EB00004C0440F551F661F771F8A95D2F7809193
:100EC000D2019091D301A091D401B091D5018A01B2
:100ED0009B01082719272A273B27C901B8011F9121
:100EE0000F910C94E6060F931F930091D20110917D
:100EF000D3012091D4013091D501602B712B822B2D
:100F0000932B1F910F910C94E6060F931F93009162
:100F1000D2011091D3012091D4013091D5016023E9
:100F20007123822393231F910F910C94E6060F9354
:100F30001F930091D2011091D3012091D4013091DF
:100F4000D50160277127822793271F910F910C9459
:100F5000E606089529E0929F800D1124E82FE6957A
:100F6000E695E695877051E001C0550F8A95EAF73E
:100F700085E0E89FF0011124E457FE4F20E030E0C7
:100F800070E04081CB01022E02C0969587950A94AD
:100F9000E2F78170819584278523842781932F5FD1
:100FA0003F4F2530310569F7089529E0929F800D64
:100FB0001124682F669566956695982F977085E041
:100FC000689FB001112440E050E080E0FB01E40F95
:100FD000F51FE457FE4F208130E0092E02C0369500
:100FE00027950A94E2F721703327042E01C0220FBF
:100FF0000A94EAF7822B4F5F5F4F4530510531F776
:101000000895BF92CF92DF92EF92FF920F931F93BA
:10101000CF93DF938C01C090D201D090D301E090A8
:10102000D401F090D5018091D6019091D701A09183
:10103000D801B091D901C82AD92AEA2AFB2ACFE1DE
:10104000D0E0D701C6010C2E04C0B695A7959795A0
:1010500087950A94D2F780FD04C0219790F7B12CB0
:1010600007C0BC2EB8018C2F0E94380F0197A9F33E
:101070008B2DDF91CF911F910F91FF90EF90DF901B
:10108000CF90BF900895CF93DF93EC010E940108A9
:10109000BE010E94380FDF91CF9108951F93CF9327
:1010A000DF93EB0190918B01992321F0CB010E94FA
:1010B000430813C0882349F0CB010E940108182F70
:1010C000682FCE010E94AA0704C0CB010E94D50759
:1010D000182FBE01812F0E94380FDF91CF911F91F1
:1010E00008951F93CF93DF93C091DA0116E08091AA
:1010F000DB01C81799F0D0E01C9FF0011D9FF00D97
:101100001124E452FE4F40815181628173818481B8
:1011100095810E948A062196C770E9CFDF91CF9111
:101120001F91089540910C0250910D0260910E02A2
:1011300070910F0280911002909111020C948A0616
:10114000EF92FF920F931F93CF93DF938091110241
:1011500082958F7009F065C080910E02882309F492
:1011600060C08091DA01F090DB0110910C020091D7
:101170000D0260910F027091100291E01F3F09F083
:1011800090E0C0910001D0910101292F96E0E92E55
:101190008F1509F446C06115710521F00F3F21F04C
:1011A00030E003C031E001C0322F90E030FD36C0A6
:1011B000E89EF001E99EF00D1124DF01A452BE4F1C
:1011C00011963C911197301329C03C91311326C0E0
:1011D00012963C911297311121C013964D915C915A
:1011E0001497461B570B4C175D07C0F480911102F2
:1011F0008F70806180931102EF51FE4F80818F705C
:10120000806180838CE092E00E940C06DF91CF9198
:101210001F910F91FF90EF900C94710801968770C9
:10122000B7CFDF91CF911F910F91FF90EF9008956D
:101230009F92AF92BF92CF92DF92EF92FF920F9365
:101240001F93CF93DF93CDB7DEB761970FB6F894B6
:10125000DEBF0FBECDBF8C0185E0F801DE011D961B
:1012600001900D928A95E1F7D8011296EC90909139
:101270000C02E0910D0220910F0230911002211515
:10128000310531F0EF3F31F481E09F3F19F403C0A5
:1012900081E001C080E0B82FB1709B2E80FD47C176
:1012A000D8014C9111965C9111971396AD90BC901A
:1012B00014978CE0C82E82E0D82EF0900E02B50173
:1012C000621B730B2091000130910101FF2009F492
:1012D000D9C0809111026217730708F095C0282FBA
:1012E000207F09F052C05E1313C0491311C0FE2CB9
:1012F000E1100EC08F708061809311020E949208ED
:10130000C6010E940C0680911102F80185834DC12F
:10131000AB2831F05F3F31F481E04F3F19F403C057
:1013200081E001C080E080FD03C081E08E2502C025
:1013300080E090E0F82FF170FF2E80FF1CC08091BC
:10134000DA012091DB0136E0821709F40BC190E04D
:10135000389FF001399FF00D1124E452FE4F618156
:10136000561306C06081461303C06281E61203C0B3
:1013700001968770E9CFFE2CEE2009F416C180910A
:10138000110281608093110254C05E1306C049139C
:1013900004C0E11002C0F80199C0C8010E947306A0
:1013A000882361F1EE2051F120911102822F829564
:1013B0008F7090E0029774F080910C0290910D0272
:1013C00098878F831986BB86AA862C87CE010796BD
:1013D0000E940C0686E0F801ACE0B2E001900D92AC
:1013E0008A95E1F70E94A0080E9492080AC05E1741
:1013F00011F1C8010E94730681112CC0C8010E941E
:101400000C06FF24F394D1C0282F207F81F77A2D7A
:10141000B98AA88A6E2D89890E947B068CE092E0A9
:101420000E940C0686E0D6011D928A95E9F70E947B
:101430009208F12CBAC04913DCCFE110DACFF801E1
:101440008583C8010E940C0686E0D6011D928A950C
:10145000E9F7ABC0EE2091F220911102822F829524
:101460008F7090E002970CF4B5CF80910C029091B0
:101470000D029A8389831B82BD82AC822E83CE01AA
:101480000196A6CF6217730708F044C0FE2CEE2029
:1014900009F4B4CF5E1330C049132EC0209111025D
:1014A00020FD21C0822F82958F70482F50E041157A
:1014B0005105C9F0F80125834F30510541F08F5F88
:1014C000982F9295907F822F8F70892B8583C801EA
:1014D0000E940C0686E0F801ACE0B2E001900D92AB
:1014E0008A95E1F73CC086E0F801ACE0B2E00190FB
:1014F0000D928A95E1F759C0C8010E9473068111C7
:1015000069CF80911102816080931102C8010E940D
:101510000C064BC07A2DB98AA88A6E2D89890E9443
:101520007B0686E0D6011D928A95E9F718C0EE2069
:1015300009F464CFC8010E947306F82E882309F4C9
:101540005DCF86E0F801ACE0B2E001900D928A95A3
:10155000E1F78CE092E00E9420030E94A0080E9424
:10156000920823C04D875E878D859E850E94430823
:10157000292F22952F70223028F49F7039F0811185
:1015800005C00BC0243028F49F7049F4805E883079
:1015900020F0C8010E940C069F2CF92C06C0D8012F
:1015A00015969C91907F91F7F8CF8F2D61960FB68D
:1015B000F894DEBF0FBECDBFDF91CF911F910F9189
:1015C000FF90EF90DF90CF90BF90AF909F900895E5
:1015D0001F93CF93DF93CDB7DEB72C970FB6F89458
:1015E000DEBF0FBECDBF4F83588769877A878B8751
:1015F0009C87CE0107960E9418098823D1F09F810D
:1016000088852A853B85232B31F08F3F31F481E09B
:101610009F3F19F403C081E001C080E080FD47C016
:101620004F81588569857A858B859C850E948A06BD
:101630003EC086E0FE013796DE01119601900D92C4
:101640008A95E1F7FF81E8856A857B8561157105DB
:1016500031F0EF3F31F481E0FF3F19F403C081E046
:1016600001C080E080FD23C02091DB0130E0C90192
:101670000196877099274091DA0150E08417950709
:10168000F1F1F983EA837D836C8396E0929FD00128
:10169000939FB00D1124A452BE4FFE0131960190CC
:1016A0000D929A95E1F78093DB010E94710816E094
:1016B0008091DA019091DB01891771F1189FC001C7
:1016C000112484529E4F0E941809882329F1E09129
:1016D000DA011E9FF0011124E452FE4F4081518136
:1016E00062817381848195810E948A068091DA01EA
:1016F00090E00196877099278093DA01D9CF0E94F4
:1017000054061092DB011092DA01ECE0F2E086E080
:10171000DF011D928A95E9F72C960FB6F894DEBF8B
:101720000FBECDBFDF91CF911F91089580911A0216
:10173000859585958595089580911A0287700895FD
:1017400090911A02977081E009F480E008958091E9
:101750002502089590912502892B809325020895F2
:1017600080959091250289238093250208951092F7
:101770002502089590912402892B809324020895D4
:1017800080959091240289238093240208951092D9
:101790002402089580911B02089508950C94CD0BA6
:1017A0000C94CE0B9091640292FD08C090911B02A4
:1017B000981721F080931B020C94D00B0895809110
:1017C0001B02882329F010921B0280E00C94D00B9E
:1017D0000895CF93DF93E0910201F091030180918E
:1017E00025028083E0910201F091030190818091B4
:1017F0002402892B808380911B02882381F0E09151
:101800000201F09103019081892B80838091020174
:10181000909103010E946B1481110E94DF0BC09113
:101820000201D091030148E050E062E172E0CE0194
:101830000E94791C892B69F088E0FE01A2E1B2E0E8
:1018400001900D928A95E1F7CE01DF91CF910C9432
:101850003414DF91CF9108950C94CD0B90916402D4
:1018600092FD10C098E0899F90011124262B2093AF
:101870001A020E940C0780911A028595859585951C
:101880000C942C0C0C940C0710921A0280E00C940F
:101890002C0C20911A028095822380931A02982F93
:1018A000977099F430E0482F082E000C550B241740
:1018B000350759F09091640292FD07C08595859592
:1018C00085950E942D070C94440C08959091640214
:1018D00092FB222720F9281769F080FB92F9909358
:1018E000640280916302909164020E94B40C82E0D1
:1018F0000C94490C08958091640282FB882780F93A
:1019000091E089270C94660C81E00C94660C80E0D1
:101910000C94660C6FEF7FEF80E090E00C94B21CAB
:1019200080E090E00E948E1C21E0893E9E4F09F0ED
:1019300020E0822F089582E090E00C94861C83E0E2
:1019400090E00C94861CCF9384E090E00E94861C6B
:10195000C82F82E290E00E94861C2C2F30E0A90163
:10196000582BCA01CF910895CF93C92F682F84E0D7
:1019700090E00E94941C6C2F82E290E0CF910C9436
:10198000941CAB01BC018FE090E00C94A61CAB0151
:10199000BC0183E190E00C94A61C60E070E0CB01F8
:1019A0000C94C70C60E070E0CB010E94C10C0C9459
:1019B000CD0C69EE7EEF80E090E00E94B21C60E00A
:1019C00082E090E00E94941C60E083E090E00E943E
:1019D000941C1092D6011092D7011092D801109247
:1019E000D90160E084E090E00E94941C60E082E213
:1019F00090E00E94941C60E085E090E00E94941CBE
:101A000060E086E090E00E94941C6FEF87E090E039
:101A10000E94941C40E050E0BA0188E090E00E94EF
:101A2000A61C60E08DE090E00E94941C40E050E035
:101A3000BA0188E190E00E94A61C60E087E190E096
:101A40000E94941C40E050E0BA018CE190E00E94BA
:101A5000A61C60E070E080E290E00E94B21C40E0D2
:101A600050E0BA0188E190E00E94A61C0C94D20CD0
:101A70000C94D90C682F8EE090E00C94941C0E947A
:101A800060156093420270934302809344029093E6
:101A9000450260933E0270933F0280934002909310
:101AA0004102089585B7806885BF85B7806885BF86
:101AB000089581E008950C94590D08950C945D0DDE
:101AC0000C945D0D0C94600D0C945D0D0C94640DE4
:101AD0000C945D0D0E94520D84E190E10E941E1451
:101AE0000E94680D0C94660D0E945E0D0C945D0DB5
:101AF0000E942E100C94BA020E944B150E942211D3
:101B00000E94780D0C94620D5F926F927F928F927B
:101B10009F92AF92BF92CF92DF92EF92FF920F937C
:101B20001F93CF93DF93CDB7DEB72A970FB6F89404
:101B3000DEBF0FBECDBF0E943711C82E81110E949B
:101B40003F0D36E2832E32E0932E00E010E0502E5F
:101B5000802F0E9452105C01F401619071904F013E
:101B60006826792661147104B1F40F5F1F4F0C30A1
:101B7000110569F78FEF89838A831B820E945415B0
:101B80008160782F9D838C8349815A816B818D81FF
:101B90000E94D6023AC08091460281FD0E945B10ED
:101BA000D12CEE24E394F12CC3018E219F21892BAB
:101BB00029F10E945B0D8823A9F0DE825F82AE20AE
:101BC000BF2081E0AB2809F480E088870E9454158B
:101BD0008160782F9A8789874E815F8168858A85A1
:101BE0000E94D602000F111FF801EA5DFD4F8081AF
:101BF0009181E826F926F182E08207C0D394EE0CA9
:101C0000FF1CF9E0DF12D0CFB0CF81E0C11001C0DE
:101C100080E02A960FB6F894DEBF0FBECDBFDF91ED
:101C2000CF911F910F91FF90EF90DF90CF90BF90D9
:101C3000AF909F908F907F906F905F9008950E94DB
:101C4000840D0C94CB02CF93DF930E943D0FEC01E7
:101C5000811522E59207E8F5811531E5930708F033
:101C6000B6C0883E910528F5803E910508F0E9C090
:101C7000883A910570F4853A910508F07AC0813070
:101C8000910509F473C008F4D9C0049708F0D9C0CD
:101C9000D5C08F3B910508F0D1C0C85AD0E0CC0F19
:101CA000DD1FCE5BDE4F0990D881C02DCE0194643C
:101CB000C9C0811540E5940708F069C0811550E45A
:101CC000950708F060C09A9581159F4108F4B9C046
:101CD000B5C0811536E5930728F5811545E59407CC
:101CE00008F092C0811554E5950708F087C0AC0153
:101CF00043705527282F26952695C115D34508F002
:101D00006CC081E090E002C0880F991F4A95E2F70D
:101D100040E2249F90011124EC01C22BD32BCE0171
:101D20009C6890C081152AE5920780F4811539E5F9
:101D3000930708F072C0811548E5940708F47EC047
:101D4000D82FCC27CE01806F906A7CC09056811529
:101D5000904208F073C08D2F8F710E94D10FDD2744
:101D6000D0628F71AE01582BCA016CC081E090E047
:101D700069C0C55AD0E0C059DE4F8881C82FD0E075
:101D8000CE0190645FC0DF70CE01906A5BC074E0EA
:101D9000969587957A95E1F7282F23703C2F33701D
:101DA00081E090E002C0880F991F3A95E2F79C68A5
:101DB000AC01522B9A019C2F9F709695969550E2FC
:101DC000959FE0011124C9018C2B9D2B3BC0D82F7E
:101DD000CC27CE01816F906A35C081E090E002C0CF
:101DE000880F991F4A95E2F750E2259F9001112430
:101DF000EC01C22BD32BCE019A6824C0D82FCC275C
:101E0000CE01846F906A1EC00E94D10F8F7190E046
:101E1000D82FCC27CE01906215C08F700E94D10FB1
:101E200094E0D695C7959A95E1F7CF70D0E0DC2F76
:101E3000CC27D0699E01282BC90104C080E090E026
:101E400001C0CE01DF91CF9108952CE6829FC001A1
:101E50001124FC0129E0729FE00DF11D1124E60F11
:101E6000F11DEE0FFF1FE852FF4F859194910895E9
:101E70000E94250F0E94230E08958238910569F172
:101E8000B0F48133910509F46DC048F489329105AD
:101E900009F463C08A32910509F469C00895853355
:101EA000910509F455C089339105B9F00895833E31
:101EB000910569F138F4803E9105B1F0823E9105BB
:101EC00009F10895863E9105A9F1873E9105B9F182
:101ED000843E910509F064C023C02091630220FD77
:101EE0004FC021FD4DC008958091630280FD44C024
:101EF0008091640280FF44C08091630284FD42C0EF
:101F000083EE4DC08091630282FF38C0F5CF80918F
:101F1000630282FD33C08091640280FD31C0ECCF4A
:101F20008091640281FF32C08091630284FD2AC0E7
:101F300087EE35C08091630283FF26C0F5CF809184
:101F4000630283FD21C08091640281FD1FC0ECCF3C
:101F50008091630285FD1CC01DC08091630285FDD8
:101F600019C016C08091630286FD16C017C080910B
:101F7000630286FD13C010C089E311C082EE0FC05A
:101F800080EE0DC080E00BC086EE09C084EE07C075
:101F900089E205C085E303C08AE201C081E390E0E5
:101FA00008959091630292FF0DC0282F2871283068
:101FB00019F4877F846006C0282F2471243011F41F
:101FC0008B7F886093FF0DC0282F2871283119F46A
:101FD000877E846106C0282F2471243111F48B7E02
:101FE00088612091640220FF0DC0382F387138308D
:101FF00019F4877F816006C0382F3171313011F4B8
:102000008E7F886021FF0DC0282F2871283119F498
:10201000877E816106C0282F2171213111F48E7EC7
:10202000886194FD877E089580E008950C948A0C61
:102030000E9437118FE39CE90197F1F700C000007F
:102040000E94371180E00E94521080FF04C00E945D
:1020500016100C94A11508950C9418100E94900C61
:10206000811102C00E94380D0E949B0C8093460291
:102070000E94A30C90936402809363020E942C1030
:102080000E949F0C682F70E080E090E00E94AC06F8
:102090006091D2017091D3018091D4019091D501CA
:1020A0000C94E406E82FF0E0EE0FFF1FE358FD4F1D
:1020B000808191810895089580EA8A95F1F70895C5
:1020C00000C008950C945C1008950C9464100C9456
:1020D00065100C9464100C946910F894E82FE29544
:1020E000EF70F0E031A1282F2F7081E090E001C067
:1020F000880F2A95EAF7982F9095932391A392A1A0
:10210000892B82A3789408950F931F93CF93DF9325
:10211000C3E7D1E089918F3F11F00E946D1081E0FB
:10212000CC37D807B9F7CCE7D1E008E811E08991BE
:102130008F3F11F00E946D100C171D07C1F7DF9142
:10214000CF911F910F910895AF92BF92DF92EF92BE
:10215000FF920F931F93CF93DF93C62FD0E0CD58FC
:10216000DE4F28812F3F09F463C08A01F62EE92E45
:10217000D82EF894E22FE295EF70F0E091A1822F33
:102180008F7021E030E001C0220F8A95EAF7892F95
:10219000822B81A382A12095282322A378940E94D8
:1021A00060108CE7A82E81E0B82EED2DFE2D9F014A
:1021B000285E3F4FE12CA80140955095D5016D91C7
:1021C0005D016F3FC9F0862F82958F7090E0DC0132
:1021D00090968C9190E06F7002C0959587956A9566
:1021E000E2F780FD09C080819181802B912B918342
:1021F0008083EE24E39406C080819181842395231B
:10220000918380833296E217F307C1F688818F3F6E
:1022100011F00E946D106E2D8F2DDF91CF911F91C7
:102220000F91FF90EF90DF90BF90AF900C946210F1
:10223000DF91CF911F910F91FF90EF90DF90BF90B2
:10224000AF9008950E94841088E1EDE7F2E0DF018D
:10225000982F1D929A95E9F7E5E6F2E0DF011D92CD
:102260008A95E9F78CE00E948C110C944502CF927C
:10227000DF92FF920F931F93CF93DF93CDB7DEB71B
:1022800068970FB6F894DEBF0FBECDBF8E010F5F0B
:102290001F4F88E1F80111928A95E9F7F12CCC24BF
:1022A000C394D12CA6016F2DC8010E94A410F394F1
:1022B000CC0CDD1CF9E0FF12F5CF48E150E0B8018D
:1022C00085E692E00E94791CFF24F394009709F4BC
:1022D000F12C892B41F088E1F801A5E6B2E00190EC
:1022E0000D928A95E1F72F2D4CE06DE772E085E6BF
:1022F00092E00E948D110E9447028F2D68960FB6C2
:10230000F894DEBF0FBECDBFDF91CF911F910F912B
:10231000FF90DF90CF9008950895FF920F931F9341
:10232000CF93DF93F82E092F162FD72FC42F2223F8
:1023300049F081E0809349020E945415909348022D
:1023400080934702809149028823D9F08091470207
:10235000909148020E946C15059798F0EF2DF02F90
:10236000A12FBD2F80E090E04C2F50E084179507FF
:1023700034F4219131912D933D930196F7CF109232
:102380004902DF91CF911F910F91FF9008950E9414
:1023900039170E947C0D0C9445170E9449170E9422
:1023A0001F0E0C9463170E94F2140E9420170E94C3
:1023B0006A0D0E94C7110E94CD110E94740DFBCFBF
:1023C000CF93DF93EC01FB018281882309F43CC1A8
:1023D000C430FDE5DF0760F4CB3F9CE5D90788F406
:1023E0009E0122503C452431310508F02EC109C020
:1023F000C236EDE5DE0729F0C63AFDE5DF0709F054
:1024000024C10E94A30C9093640280936302C131A3
:102410008CE5D80709F4C6C008F042C0C930ECE525
:10242000DE0709F49BC000F5C5308CE5D80709F438
:1024300085C078F4C330ECE5DE0709F478C008F015
:102440007AC0C230DC4509F0F5C08091630281603A
:10245000EFC0C7309CE5D90709F478C008F07AC00E
:10246000809163028061E4C0CD30FCE5DF0709F4B0
:1024700087C058F4CB309CE5D90709F479C008F03F
:102480007BC08091630288606FC0CF30FCE5DF07BE
:1024900009F480C008F082C080916302877FC8C0C1
:1024A000CE3F9CE5D90709F471C000F5C531FCE5C4
:1024B000DF0709F485C068F4C3319CE5D90709F446
:1024C00075C008F095C00E945406809163028F7712
:1024D000AFC0CC3FFCE5DF07A9F108F054C0CB3F0B
:1024E000DC4509F0A7C08091640240C0C230EDE530
:1024F000DE0709F489C058F4C1158DE5D80709F441
:102500005AC008F069C08091640282602FC0C23650
:10251000EDE5DE0709F47CC0C63AFDE5DF0709F406
:1025200081C0C330DD4509F085C080E06EC0809178
:10253000630282607DC08091630216C08091630255
:10254000886076C08091640282604FC0809163028F
:1025500080626EC08091630280646AC00E945406EB
:1025600080916302806864C0846062C081603DC005
:10257000809163028E7F5CC0809163028D7F58C022
:102580008091630216C08091640218C08091640239
:102590008D7F2BC0809163028F7E4AC08091630241
:1025A0008F7D46C0809163028F7B42C08091630221
:1025B000877F8B7F3DC0809164028D7F8E7F15C0A9
:1025C0008091630282FB222720F991E0922790FB01
:1025D00082F990FB83F92CC080916402982F90952A
:1025E00091708E7F892B90FB81F98093640222C0C9
:1025F0000E9454068091630287FB222720F991E014
:10260000922790FB87F914C081E00E943A0D12C016
:102610008091630284FB222720F991E0922790FBAE
:1026200084F906C080916302982F909590FB80F901
:102630008093630280916302909164020E94B40CC3
:102640000E94540680E001C081E0DF91CF9108959F
:10265000CF93DF9386319C4541F5EB010E94A70B98
:10266000982F8A812091020130910301882379F00B
:102670009A7A81E009F480E080934A02911102C0C5
:1026800069E201C065E3C9010E94AD140AC08091EE
:102690004A02811102C069E201C065E3C9010E94DA
:1026A000AF140E94E90B80E001C081E0DF91CF917F
:1026B00008950F931F93CF93DF93C42FD22FFC0164
:1026C00082818823C9F040934D020E945415909353
:1026D0004C0280934B0280E28C0F883008F057C088
:1026E000C77081E001C0880FCA95EAF7DF91CF91EA
:1026F0001F910F910C94C00380914D02481330C07C
:1027000080914B0290914C020E946C15883C91057F
:1027100038F510E21D0FCD17B9F080E28C0F88302C
:1027200040F4C77081E001C0880FCA95EAF70E94A3
:10273000C703183028F581E09D2F977001C0880FDE
:102740009A95EAF70E94C003802F0E94B7031830C1
:10275000F0F4D77081E001C0880FDA95EAF70AC07B
:1027600080E28C0F883098F4C77081E001C0880F38
:10277000CA95EAF7DF91CF911F910F910C94C7038F
:10278000802FDF91CF911F910F910C94B703DF91B0
:10279000CF911F910F9108950F939C01CB01243F7E
:1027A0004CE5340731F188F4293DFCE53F07D9F0C9
:1027B0002A3D4CE5340779F1283D3C45A9F506E270
:1027C00021EE41EE68ED7CE52BC0263FFCE53F079E
:1027D000E1F0A8F0273F3C4539F507E225EE46EE4B
:1027E00067EF7CE51DC007E225EE45EE69ED7CE56F
:1027F00017C006E221EE40EE64EF7CE511C007E26F
:1028000025EE44EE65EF7CE50BC006E221EE42EEDC
:1028100066EF7CE505C008E221E045EE6AED7CE567
:102820000E94591380E008C0FC018281882319F0BE
:1028300010924D0201C081E00F910895909389019B
:1028400080938801089590935302809352020895D3
:10285000E0915202F0915302309721F00190F08103
:10286000E02D099480E00895E0915202F091530226
:10287000309721F00280F381E02D09940895209192
:102880005002309151022817390771F0909351028C
:1028900080935002E0915202F0915302309721F060
:1028A0000680F781E02D0994089520914E02309121
:1028B0004F022817390771F090934F0280934E0210
:1028C000E0915202F0915302309721F00084F1859B
:1028D000E02D09940895FC01329697E080E0915034
:1028E00029F021912223D9F38F5FF9CF0895662330
:1028F00049F0FC01329608962191621729F0E817F9
:10290000F907D1F780E0089581E008959C01FC016A
:1029100032969FEF80E04191461789F09F3F19F46E
:10292000411101C0982F8F5F8630A9F79F3F39F082
:10293000F901E90FF11D97FDFA9562830895089555
:102940009C012A5F3F4FFC014281461301C0128265
:10295000019682179307B9F708950C9486140C9486
:10296000A014029626E0FC0111922A95E9F7089539
:1029700008950C94B81483E0809354020C94B91415
:10298000811102C081E001C082E0809354020C9466
:10299000B9140C94C01481E0809354020C94B914BF
:1029A0000C94CB1408950C94D2140C94D3140C945E
:1029B000D2140C94D2140C94D214CF930E94D91434
:1029C0000E9437110E94D714C0E08C2F0E94521031
:1029D000892B29F4CF5FCC30C1F780E001C081E0C2
:1029E000CF91089508951F920F920FB60F92112460
:1029F0008F939F93AF93BF9380915502811113C022
:102A00008091950290919602A0919702B0919802C0
:102A10004196A11DB11D8093950290939602A093BB
:102A20009702B0939802BF91AF919F918F910F90B1
:102A30000FBE0F901F90189580919D02843031F148
:102A40000E94AB021092550220E488E190E00FB69C
:102A5000F894A895809360000FBE2093600083B720
:102A6000817F846083BF83B7816083BF78948895BA
:102A700083B78E7F83BF0FB6F894A89580916000CE
:102A8000886180936000109260000FBE08950E94DC
:102A900054060C94AF0282E084BD93E095BD9AEF9A
:102AA00097BD80936E0008952FB7F894809195029A
:102AB00090919602A0919702B09198022FBF08952D
:102AC0002FB7F894609195027091960280919702C9
:102AD000909198022FBF08959C014FB7F894809170
:102AE000950290919602A0919702B09198024FBFE3
:102AF000821B930B089578941F920F920FB60F923A
:102B000011248F939F93AF93BF93809195029091DF
:102B10009602A0919702B09198020196A11DB11D55
:102B20008093950290939602A0939702B093980297
:102B3000BF91AF919F918F910F900FBE0F901F90FB
:102B4000189581E08093E00080E28093D800109295
:102B5000C9008FE19EE40197F1F700C0000087E013
:102B600090EBDC018093A6029093A702A093A802A9
:102B7000B093A9029CE088E10FB6F894A8958093E1
:102B800060000FBE90936000FFCF809161020895B6
:102B90000895CF93DF9321E02093E9002FEF309148
:102BA000E800215035FD06C035ED3A95F1F70000FB
:102BB0002111F5CF2091E80025FF14C0EC0140E081
:102BC00050E068E070E00E94D5178091E8008E77B1
:102BD0008093E80088E0FE01A9E5B2E001900D9243
:102BE0008A95E1F7DF91CF91089580935602709313
:102BF00058026093570280919D02843001F582E073
:102C00008093E9008FEF9091E800815095FD06C018
:102C100095ED9A95F1F700008111F5CF8091E800CC
:102C200085FF0DC040E050E063E070E086E592E093
:102C30000E94D5178091E8008E778093E800089570
:102C4000BC0184E00C94F515BC0183E00C94F515EF
:102C5000089580919C02811109C00E9466190E940A
:102C6000C3198091E20084608093E200089510927D
:102C70009C0208950C94D0146091990281E0611136
:102C800001C080E00C94BB1490919D0281E09430CF
:102C900009F080E0609199020C94C01442E061EC6C
:102CA00081E00E94DF1842E261EC82E00E94DF18BE
:102CB00090919D0281E0943009F080E0609199024A
:102CC0000C94C91480919F02833009F461C030F4E0
:102CD000813071F0823009F49AC008958A3009F485
:102CE00086C08B3009F46CC0893009F0A8C020C0C0
:102CF00080919E02813A09F0A2C08091E800877F0E
:102D00008093E8008091A2029091A302892B21F484
:102D100068E089E592E003C060E080E090E070E068
:102D20000E9420188091E8008B778093E800089536
:102D300080919E02813209F082C08091A20290911E
:102D4000A302029708F07BC08091E800877F809300
:102D5000E8008091E80082FD05C080919D0281110C
:102D6000F8CF6DC02091F3008091F20090E0922B9B
:102D7000029731F48091F100813011F0863021F416
:102D80008091F100809361028091E8008B7753C0BD
:102D900080919E02813A09F052C08091A2029091E6
:102DA000A302892B09F04BC08091E800877F8093B4
:102DB000E8008091E80080FFFCCF8091100136C0D0
:102DC00080919E028132D9F58091A2029091A30256
:102DD000892BA9F58091E800877F8093E8000E9405
:102DE00014198091A002809310010C9454068091D4
:102DF0009E02813221F58091E800877F8093E80070
:102E00000E9414198091A10280936202089580911A
:102E10009E02813AA1F48091E800877F8093E800C8
:102E20008091E80080FFFCCF809162028093F100E6
:102E30008091E8008E778093E8000C94141908952F
:102E400084B7877F84BF0FB6F894A89580916000FF
:102E5000886180936000109260000FBE90E080E86F
:102E60000FB6F89480936100909361000FBE0C94AC
:102E7000CB140E9466190E94C319E2EEF0E0808133
:102E80008460808378940C94581C84E091E00C94C6
:102E9000231480919D028530A9F480919D02853094
:102EA00079F40E941C1580919B028823B1F30E9443
:102EB000DD14882391F30E94BF170E945406EDCFC2
:102EC0000C944715089508950C946617292F3327FD
:102ED00023303105C9F060F42130310581F0223012
:102EE000310509F044C08BE390E022EB32E043C0AF
:102EF00021323105E1F02232310549F138C082E159
:102F000090E02DEE32E037C099278130910549F0ED
:102F100028F0029761F5E8E8F2E005C0EEEAF2E099
:102F200002C0EAE9F2E0849190E09F0124C06115BB
:102F3000710541F061307105D1F489E090E02DED2B
:102F400032E019C089E090E024EC32E014C0611551
:102F5000710541F06130710551F482E390E02FEF8B
:102F600032E009C080E490E021E333E004C080E077
:102F700090E020E030E0FA0131832083089580E181
:102F800089BD82E189BD09B400FEFDCF8091D800E2
:102F90008F7D8093D8008091E00082608093E00074
:102FA0008091E00081FDFCCF0895CF92DF92EF92F7
:102FB000FF920F931F93CF93DF93EC018B017A0164
:102FC0000E943319811133C0E114F10439F0F70183
:102FD00080819181081B190BC80FD91FC12CD12CDE
:102FE0000115110519F18091E80085FD16C0809149
:102FF000E8008E778093E800E114F10449F0F701CE
:1030000080819181C80ED91ED182C08285E00FC017
:103010000E943319882321F30AC089918093F1001B
:1030200001501109FFEFCF1ADF0ADACF80E0DF91FC
:10303000CF911F910F91FF90EF90DF90CF90089567
:103040002091A4023091A5022617370748F0611598
:10305000710539F42091E8002E772093E80001C033
:10306000B901FC0120E06115710579F180919D02A3
:103070008823F1F18530F1F18091E80083FD3CC0B7
:103080008091E80082FD2EC08091E80080FFEBCFA8
:103090002091F3008091F20090E0922B6115710570
:1030A00051F08830910538F421912093F10061505E
:1030B00071090196F3CF21E0089709F020E0809193
:1030C000E8008E778093E800CECF2111CFCF0AC0E1
:1030D00080919D02882361F0853061F08091E80045
:1030E00083FD0AC08091E80082FFF2CF80E008955E
:1030F00082E0089583E0089581E008952091A4027C
:103100003091A5022617370748F06115710539F48B
:103110002091E8002E772093E80001C0B901FC015E
:1031200020E06115710591F180919D02882309F4D9
:1031300040C0853009F43FC08091E80083FD3DC068
:103140008091E80082FD2FC08091E80080FFE9CFE8
:103150002091F3008091F20090E0922B61157105AF
:1031600059F08830910540F424912093F100319674
:10317000615071090196F2CF21E0089709F020E033
:103180008091E8008E778093E800CBCF2111CCCFDF
:103190000AC080919D02882361F0853061F08091A2
:1031A000E80083FD0AC08091E80082FFF2CF80E052
:1031B000089582E0089583E0089581E00895982FAE
:1031C000973068F59093E900981739F07091EC000A
:1031D0002091ED005091F00003C0242F762F50E095
:1031E00021FD02C09F5FECCF3091EB003E7F30931A
:1031F000EB003091ED003D7F3093ED003091EB001E
:1032000031603093EB007093EC002093ED0050930D
:10321000F0002091EE0027FDE5CF80E008958F704B
:103220008093E90081E0089580919E0287FF11C09C
:103230008091E80082FD05C080919D028111F8CF48
:1032400011C08091E8008B770BC080919D0288238C
:1032500049F08091E80080FFF8CF8091E8008E77F8
:103260008093E80008952091E4003091E50095E610
:103270004091EC00842F817040FF23C08091E800D2
:1032800080FD1DC080919D02882399F0853099F0C2
:103290008091EB0085FD11C04091E4005091E50064
:1032A0002417350729F3915011F09A01E1CF84E0FA
:1032B000089582E0089583E0089581E0089580E014
:1032C00008954091E80042FFDDCF08950E94D4198F
:1032D0000E94DC19E0EEF0E0808181608083E8EDFF
:1032E000F0E080818F77808319BCA7EDB0E08C91EE
:1032F0008E7F8C9380818F7E808310929C020895B4
:103300000F931F93CF93DF930E94D4190E94DC196F
:10331000C8EDD0E088818F77888388818068888332
:1033200088818F7D888319BC10929D02109299022A
:1033300010929B0210929A0200EE10E0F801808138
:103340008B7F808388818160888342E060E080E0B9
:103350000E94DF18E1EEF0E080818E7F8083E2EE54
:10336000F0E0808181608083808188608083F801C3
:1033700080818E7F8083888180618883DF91CF9177
:103380001F910F910895E8EDF0E080818F7E80839A
:10339000E7EDF0E080818160808384E082BF81E09E
:1033A00080939C020C948019E8EDF0E080818E7F80
:1033B00080831092E20008951092DA001092E100EA
:1033C00008951F920F920FB60F9211242F933F93DF
:1033D0004F935F936F937F938F939F93AF93BF931D
:1033E000EF93FF938091E10082FF0BC08091E20098
:1033F00082FF07C08091E1008B7F8093E1000E94F3
:10340000571C8091DA0080FF1FC08091D80080FF98
:103410001BC08091DA008E7F8093DA008091D90002
:1034200080FF0DC080E189BD82E189BD09B400FE45
:10343000FDCF81E080939D020E94291605C019BC32
:1034400010929D020E9437168091E10080FF19C002
:103450008091E20080FF15C08091E2008E7F809312
:10346000E2008091E20080618093E2008091D800C8
:1034700080628093D80019BC85E080939D020E94F1
:103480003C168091E10084FF30C08091E20084FF0F
:103490002CC080E189BD82E189BD09B400FEFDCF69
:1034A0008091D8008F7D8093D8008091E1008F7E3D
:1034B0008093E1008091E2008F7E8093E200809112
:1034C000E20081608093E20080919902882311F0EC
:1034D00084E007C08091E30087FD02C081E001C065
:1034E00083E080939D020E9444168091E10083FF57
:1034F00029C08091E20083FF25C08091E100877F91
:103500008093E10082E080939D0210929902809165
:10351000E1008E7F8093E1008091E2008E7F8093B6
:10352000E2008091E20080618093E20042E060E08E
:1035300080E00E94DF188091F00088608093F000A6
:103540000E943A16FF91EF91BF91AF919F918F9199
:103550007F916F915F914F913F912F910F900FBE8F
:103560000F901F9018951F920F920FB60F92112473
:103570002F933F934F935F936F937F938F939F937B
:10358000AF93BF93CF93DF93EF93FF93C091E90085
:10359000CF708091EC00D82FD17080FDD0E81092D0
:1035A000E9008091F000877F8093F00078940E947A
:1035B000F71A1092E9008091F00088608093F00083
:1035C000CD2BCF70C093E900FF91EF91DF91CF91A8
:1035D000BF91AF919F918F917F916F915F914F912B
:1035E0003F912F910F900FBE0F901F9018951F9332
:1035F000CF93DF93CDB7DEB7AA970FB6F894DEBFAF
:103600000FBECDBFEEE9F2E08091F100819322E0A0
:10361000E63AF207C9F70E9462168091E80083FF3C
:103620002EC180919E0290919F02492F50E04A3016
:10363000510508F024C1FA01EE59FF4F0C94731C98
:10364000803821F0823809F01AC108C080919A02AE
:1036500090919B02992389F082600FC08091A20211
:103660008F70873008F00BC18093E9008091EB00E8
:1036700085FB882780F91092E9009091E800977FF8
:103680009093E8008093F1001092F100D1C0282FB0
:103690002D7F09F0F4C0882319F0823061F0EFC06B
:1036A0008091A002813009F0EAC0933009F080E0F7
:1036B00080939B022EC08091A00281112AC080912C
:1036C000A2028F702FEF280F263008F0D8C0809309
:1036D000E9002091EB0020FF1CC0933021F4809181
:1036E000EB00806214C09091EB0090619093EB002E
:1036F00021E030E0A90102C0440F551F8A95E2F78E
:103700004093EA001092EA008091EB008860809379
:10371000EB001092E9008091E800877F8093E80039
:103720000E941419ACC08111AAC01091A0021F7789
:103730008091E3008078812B8093E3008091E80002
:10374000877F8093E8000E9414198091E80080FF31
:10375000FCCF8091E30080688093E300111102C0E8
:1037600082E001C083E080939D0289C0805882304E
:1037700008F085C08091A0029091A1028C3D53E099
:10378000950779F583E08A838AE289834FB7F894B5
:10379000DE01139620E03EE051E2E32FF0E050938B
:1037A0005700E49120FF03C0E295EF703F5FEF7098
:1037B0008E2F90E0EA3010F0C79601C0C0968D932E
:1037C0009D932F5F243149F74FBF8091E800877F99
:1037D0008093E8006AE270E0CE0101960E94201812
:1037E00016C06091A2027091A302AE014F5F5F4FBD
:1037F0000E946417BC01892B09F441C09091E80034
:10380000977F9093E80089819A810E947E18809129
:10381000E8008B778093E80032C0803881F5809192
:10382000E800877F8093E800809199028093F100FF
:103830008091E8008E7772CF811121C08091A00223
:103840009091A10299270297D4F48091E800877F94
:103850008093E8008091A002809399020E9414193D
:1038600080919902811106C08091E30087FD02C01A
:1038700081E001C084E080939D020E944E168091F9
:10388000E80083FF0AC08091E800877F8093E8000A
:103890008091EB0080628093EB00AA960FB6F894BB
:1038A000DEBF0FBECDBFDF91CF911F910895089568
:1038B000CF9380919D028823A1F0C091E900CF7041
:1038C0009091EC00892F817090FD80E8C82B1092B8
:1038D000E9008091E80083FD0E94F71ACF70C09341
:1038E000E900CF910895EE0FFF1F0590F491E02DB0
:1038F0000994FB01DC0104C08D910190801921F431
:1039000041505040C8F7881B990B0895F999FECF94
:1039100092BD81BDF89A992780B50895A8E1B0E0DD
:1039200042E050E00C94BA1C262FF999FECF92BDCC
:1039300081BDF89A019700B4021639F01FBA20BD74
:103940000FB6F894FA9AF99A0FBE08950396272FA6
:103950000E94951C0E94941C252F0E94951C242FC8
:103960000C94951C0196272F0E94951C0C94941C76
:10397000DC01CB01FC01F999FECF06C0F2BDE1BD2F
:10398000F89A319600B40D9241505040B8F708951E
:04399000F894FFCFD9
:10399400C8001C02C515C915281624162016C815FA
:1039A40001E200E900EA00B500B600B700CD0083EB
:1039B40001CC008A019201940121022302240225F0
:1039C40002260227022A02B300B4006F00700081AD
:1039D4008283E200E900EA00B500B600B700CD003A
:1039E4008301CC008A019201940121022302240262
:1039F4002502260227022A02B300B4006F007000D9
:103A0400818283F0F1F4F5F6F76795933130333220
:083A14009037929135346636BB
:00000001FF
